:100000000C942A000C94CD0518950000189500005A
:10001000189500001895000018950000189500002C
:10002000189500001895000018950000189500001C
:10003000189500001895000018950000189500000C
:1000400018950000189500001895000018950000FC
:10005000189500008FE58DBFC0E4E8E34E2E88E0E0
:100060008EBFD8E0F8E05F2EEEEFF7E0A0E6B0E05C
:1000700088278D933197E9F787E689B980E080BDBD
:1000800088E18AB90E941D07662486E880BD00E4E5
:1000900012E42FE030E0A0E6B0E00D931D932D9325
:1000A0003C938CE00E9471078FEF8ABB80E087BB96
:1000B00080E08FBD82E08EBD789400E010E020E00B
:1000C00030E0A1ECB1E00D931D932D933C93ADEA8C
:1000D000B1E0E8E2F9E10E94420AA9EAB1E0ECE20B
:1000E000F9E10E94420AA5EBB1E0E0E3F9E10E94E8
:1000F000420AA1EBB1E0E4E3F9E10E94420AA1ED7A
:10010000B0E0E8E3F9E10E94420AA5EDB0E0ECE3DB
:10011000F9E10E94420AA8E9B0E0E0E4F9E10E94B6
:10012000420AA0E9B0E0E4E4F9E10E94420AA4E94D
:10013000B0E0E8E4F9E10E94420A0E9402078FE77A
:1001400011E00E941107ECE5F9E10E94FB068BE744
:100150000E946B07EEE6F9E10E94FB0683E911E0DD
:100160000E941107E0E7F9E10E94FB068FEB11E026
:100170000E941107EEE7F9E10E94FB0683ED11E012
:100180000E941107E2E9F9E10E94FB06E3E0F0E0DA
:100190000E94140781E08093D00082E08EBD80E051
:1001A00090E090934D0080934C008BB780648BBFA0
:1001B000A0EDB0E08C91E4EFF1E0ABE30E94540AD3
:1001C00084EF91E00E949E0782E08093D00082E05D
:1001D0008EBD80E090E090934D0080934C008BB7F3
:1001E00080648BBFA0EDB0E08C91E4EFF1E0ABE375
:1001F0000E94540A84EF91E00E949E0783E080935E
:10020000D00082E08EBD80E090E090934D0080931E
:100210004C008BB780648BBFA0EDB0E08C91E4EF15
:10022000F1E0ABE30E94540AE4E6F0E00E94B20879
:10023000ECE4F9E10E94180A0E94210A11F00C94E2
:1002400023010C94C806E8E6F0E00E94B208ECE452
:10025000F9E10E94180A0E94210A11F00C9432015F
:100260000C94C806ECE6F0E00E94B208ECE4F9E178
:100270000E94180A0E94210A11F00C9441010C946A
:10028000C806E4E6F0E00E94B208E0E5F9E10E9469
:10029000180A0E94210A18F011F00C9451010C94D4
:1002A00053010C94C806E8E6F0E00E94B208E0E5CD
:1002B000F9E10E94180A0E94210A18F011F00C942A
:1002C00063010C9465010C94C806ECE6F0E00E9412
:1002D000B208E0E5F9E10E94180A0E94210A18F02C
:1002E00011F00C9475010C9477010C94C806E4E5A8
:1002F000F9E10E94180AE4E6F0E00E94B2080E94C8
:100300003A0CEDE0F0E0A0E7B0E00E94460BE4E537
:10031000F9E10E94180AE8E6F0E00E94B2080E94A3
:100320003A0CEDE0F0E0A4E7B0E00E94460BE4E513
:10033000F9E10E94180AECE6F0E00E94B2080E947F
:100340003A0CEDE0F0E0A8E7B0E00E94460BE4E5EF
:10035000F9E10E94180AE0E9F0E00E94B2080E9468
:100360003A0CEDE0F0E0ACE9B0E00E94460BE4E5C9
:10037000F9E10E94180AE4E9F0E00E94B2080E9444
:100380003A0CEDE0F0E0A0EAB0E00E94460BE0E7B6
:10039000F0E00E94B708ECE9F0E00E94B2080E9489
:1003A000AE09EDE0F0E0ACE7B0E00E94460BE4E718
:1003B000F0E00E94B708ECE7F0E00E94B2080E946B
:1003C000BD09EDE0F0E0ACE7B0E00E94460BE4E5EB
:1003D000F9E10E94180AECE7F0E00E94B2080E94DE
:1003E0002709EDE0F0E0ACE7B0E00E94460BE0E961
:1003F000F0E00E94B708ECE7F0E00E94B2080E942B
:100400002709EDE0F0E0ACE7B0E00E94460BE8E73A
:10041000F0E00E94B708E0EAF0E00E94B2080E9413
:10042000AE09EDE0F0E0A8EAB0E00E94460BE4E798
:10043000F0E00E94B708E8EAF0E00E94B2080E94EB
:10044000BD09EDE0F0E0A8EAB0E00E94460BE4E56B
:10045000F9E10E94180AE8EAF0E00E94B2080E945E
:100460002709EDE0F0E0A8EAB0E00E94460BE4E9DD
:10047000F0E00E94B708E8EAF0E00E94B2080E94AB
:100480002709EDE0F0E0A0E8B0E00E94460BE4E5CB
:10049000F9E10E94180AECE7F0E00E94B2080E941D
:1004A0003A0CEDE0F0E0A8E8B0E00E94460BE4E58D
:1004B000F9E10E94180AE0E8F0E00E94B2080E9408
:1004C0003A0CEDE0F0E0ACE8B0E00E94460BE8E862
:1004D000F0E00E94B708E4E7F0E00E94B2080E9452
:1004E000AE09EDE0F0E0A8EAB0E00E94460BE8E8D3
:1004F000F0E00E94B708E8EAF0E00E94B2080E942B
:10050000AE09EDE0F0E0A8EAB0E00E94460BECE8AE
:10051000F0E00E94B708E8EAF0E00E94B2080E940A
:10052000AE09EDE0F0E0A8EAB0E00E94460BE8EA90
:10053000F0E00E94720CEDE0F0E0A4E8B0E00E9470
:10054000460BE4E8F0E00E94B708E8E9F0E00E941A
:10055000B2080E94AE09EDE0F0E0A4E8B0E00E942D
:10056000460B0E9402078FE711E00E941107E4EAA0
:10057000F9E10E94FB06A0E2B8E0AF93BF93ECE77D
:10058000F0E00E94B2080E94AD0711E003E0BF91C5
:10059000AF910E946C0AE0E2F8E0A0E2B8E00E94AD
:1005A000410B0E94F306E8EAF9E10E94FB0683E9A9
:1005B00011E00E941107EAEAF9E10E94FB06A0E2BD
:1005C000B8E0AF93BF93E0E8F0E00E94B2080E9469
:1005D000AD0711E003E0BF91AF910E946C0AE0E229
:1005E000F8E0A0E2B8E00E94410B0E94F306E8EABE
:1005F000F9E10E94FB068FEB11E00E941107EEEA81
:10060000F9E10E94FB06A0E2B8E0AF93BF93E4E8F3
:10061000F0E00E94B2080E94AD0711E003E0BF9134
:10062000AF910E946C0AE0E2F8E0A0E2B8E00E941C
:10063000410B0E94F306E8EAF9E10E94FB068FE70E
:100640001CE00E941107E2EBF9E10E94FB06A0E228
:10065000B8E0AF93BF93E4E6F0E00E94B2080E94D6
:10066000AD0711E003E0BF91AF910E946C0AE0E298
:10067000F8E0A0E2B8E00E94410B0E94F306E8EA2D
:10068000F9E10E94FB0683E918E10E941107E6EBFD
:10069000F9E10E94FB06A0E2B8E0AF93BF93E8E661
:1006A000F0E00E94B2080E94AD0711E003E0BF91A4
:1006B000AF910E946C0AE0E2F8E0A0E2B8E00E948C
:1006C000410B0E94F306E8EAF9E10E94FB068FEB7A
:1006D0001CE00E941107EAEBF9E10E94FB06A0E290
:1006E000B8E0AF93BF93ECE6F0E00E94B2080E943E
:1006F000AD0711E003E0BF91AF910E946C0AE0E208
:10070000F8E0A0E2B8E00E94410B0E94F306E8EA9C
:10071000F9E10E94FB0683ED11E00E941107EEEB68
:10072000F9E10E94FB06A0E2B8E0E4ECF0E00E94F0
:10073000CF0A0E94F306E2ECF9E10E94FB06A0E278
:10074000B8E0E8ECF0E00E94CF0A0E94F306E2EC89
:10075000F9E10E94FB06A0E2B8E0ECECF0E00E94B8
:10076000CF0A0E94F306E4E9F0E00E94B708E0E84F
:10077000F0E00E94B2080E942709EDE0F0E0A0E856
:10078000B0E00E94460BE0E9F0E00E94B708ECE719
:10079000F0E00E94B2080E942709EDE0F0E0ACE72B
:1007A000B0E00E94460BECE7F0E00E94B708E8E5F5
:1007B000F9E10E940F0A0E94AE09EDE0F0E0ACE71B
:1007C000B0E00E94460BE1EBF1E00E94B708E0E8E0
:1007D000F0E00E94B2080E947D09EDE0F0E0A0E8A0
:1007E000B0E00E94460BE5EBF1E00E94B708ECE7B1
:1007F000F0E00E94B2080E947D09EDE0F0E0ACE775
:10080000B0E00E94460BE9EAF1E00E94B708E0E898
:10081000F0E00E94B2080E94BD09EDE0F0E0A0E81F
:10082000B0E00E94460BEDEAF1E00E94B708ECE769
:10083000F0E00E94B2080E94BD09EDE0F0E0ACE7F4
:10084000B0E00E94460BA9EDB0E0E4ECF9E10E94B3
:10085000A208A9EDB0E00E94D606E1ECF1E00E940A
:10086000CF0AA9EDB0E00E94D606ECECF9E10E94B7
:10087000A208A9EDB0E00E94D606ECE7F0E00E94E5
:10088000B2080E94AD07A9EDB0E00E94D606E2EDE5
:10089000F9E10E94A208A9EDB0E00E94D606E0E8C6
:1008A000F0E00E94B2080E94AD07A9EDB0E00E94FE
:1008B000D606E6EDF9E10E94A208AEE3B1E0E8EF6A
:1008C000F9E10E94A208AEE3B1E00E94D606E1EC95
:1008D000F1E00E94CF0AAEE3B1E00E94D606E0E06C
:1008E000FAE10E94A208AEE3B1E00E94D606ECE76E
:1008F000F0E00E94B2080E94AD07AEE3B1E00E94B2
:10090000D606E2EDF9E10E94A208AEE3B1E00E9452
:10091000D606E0E8F0E00E94B2080E94AD07AEE320
:10092000B1E00E94D606E8E0FAE10E94A208AEE338
:10093000B1E00E94D606ECECF1E00E94CC0AAEE3F6
:10094000B1E00E94D606ECE0FAE10E94A208AEE314
:10095000B1E00E94D606EAECF1E00E94CC0AAEE3D8
:10096000B1E00E94D606EEE0FAE10E94A20880E023
:100970008093A30181E08093C501A9EDB0E00E94BE
:100980005B0B482F0091C501041718F011F00C946F
:10099000E7048091C501E9EDF0E001E00A93A7EAE0
:1009A000B1E00E944C0B0091A3010F93A7EAB1E0C4
:1009B0008C91482F0F910427A3EAB1E00C93A5EC8A
:1009C000B1E08C918F5F8C9310F40C94BD04A4EA79
:1009D000B1E0E3EAF1E00E94250BEAE1FAE10E94CE
:1009E000E506A9EDB0E00E94DF06ECE1FAE10E9425
:1009F000E506A4EAB1E00E94DF060E94EC0680E072
:100A00008093A30181E08093C501AEE3B1E00E9431
:100A10005B0B482F0091C501041718F011F00C94DE
:100A20002F058091C501EEE3F1E001E00A93A7EA0A
:100A3000B1E00E944C0B0091A3010F93A7EAB1E033
:100A40008C91482F0F910427A3EAB1E00C93A5ECF9
:100A5000B1E08C918F5F8C9310F40C940505A4EA9F
:100A6000B1E0E3EAF1E00E94250BEAE1FAE10E943D
:100A7000E506AEE3B1E00E94DF06ECE1FAE10E9498
:100A8000E506A4EAB1E00E94DF060E94EC06A1ECB4
:100A9000B1E00D911D912D913C9141E050E060E05D
:100AA00070E00E94B40AA1ECB1E00D931D932D9368
:100AB0003D9341E050E060E070E0A1ECB1E00D91C9
:100AC0001D912D913C910E94B90A11F00C946E0574
:100AD000EEE1FAE10E94E5060E94EC0641E050E0FA
:100AE00060E070E0A1ECB1E00D911D912D913C9181
:100AF0000E94B90A11F00C948305E6E5FAE10E9420
:100B0000E5060E94EC0641E050E060E070E0A1ECF8
:100B1000B1E00D911D912D913C910E94B90A11F007
:100B20000C949805ECE9FAE10E94E5060E94EC06B7
:100B300041E050E060E070E0A1ECB1E00D911D916A
:100B40002D913C910E94B90A11F00C94AD05E2EE92
:100B5000FAE10E94E5060E94EC0649E050E060E000
:100B600070E0A1ECB1E00D911D912D913C910E949E
:100B7000B90A0CF002C00C94C70500E010E020E0B8
:100B800030E0A1ECB1E00D931D932D933C9384EFE5
:100B900091E00E949E070C94CA000F921F922F9220
:100BA0003F924F925F927F92AF92BF920F931F93AB
:100BB0002F933F934F935F936F937F938F939F9365
:100BC000AF93BF93CF93DF93EF93FF938FB78F9341
:100BD0008EB5887F8EBD8BB78F7B8BBF80E0E4EFB7
:100BE000F1E0ABE30E94540A0091D000013011F013
:100BF0000C943106ACE4B0E08D919C91A4ECB0E093
:100C00008D939D9388278D938C93ECE4F0E0D190A5
:100C1000E080FF2400270E94D608A4E6B0E00E94EE
:100C20000709E1EDF0E00E94B708E4E6F0E00E9479
:100C3000B2080E94AE09EDE0F0E0A4E6B0E00E9448
:100C4000460BE5EDF0E00E94B708E4E6F0E00E9414
:100C5000B2080E942709EDE0F0E0A4E6B0E00E94AF
:100C6000460B0091D000023011F00C946E06ACE4FB
:100C7000B0E08D919C91A8ECB0E08D939D93882776
:100C80008D938C93ECE4F0E0D190E080FF2400277A
:100C90000E94D608A8E6B0E00E940709E1EDF0E066
:100CA0000E94B708E8E6F0E00E94B2080E94AE0990
:100CB000EDE0F0E0A8E6B0E00E94460BE5EDF0E0E4
:100CC0000E94B708E8E6F0E00E94B2080E942709F7
:100CD000EDE0F0E0A8E6B0E00E94460B0091D00005
:100CE000033011F00C94AB06ACE4B0E08D919C9114
:100CF000ACECB0E08D939D9388278D938C93ECE4BE
:100D0000F0E0D190E080FF2400270E94D608ACE6F6
:100D1000B0E00E940709E1EDF0E00E94B708ECE6C0
:100D2000F0E00E94B2080E94AE09EDE0F0E0ACE60F
:100D3000B0E00E94460BE5EDF0E00E94B708ECE65B
:100D4000F0E00E94B2080E942709EDE0F0E0ACE676
:100D5000B0E00E94460B8F918FBFFF91EF91DF9122
:100D6000CF91BF91AF919F918F917F916F915F9143
:100D70004F913F912F911F910F91BF90AF907F9016
:100D80005F904F903F902F901F900F90189508956F
:100D90000E940207E8E1FBE10E94FB06E2E0F0E0CE
:100DA0000E9414070C94CA00F894FFCF8F938D9182
:100DB0008823E9F711978F910895A0E2B8E08D910B
:100DC000882311F00CD0FBCF08950E940B0A802DD0
:100DD00011F005D0FACF08958DE001D08AE05D9B37
:100DE000FECF8CB90895A0E2B8E08D91882311F070
:100DF00072D0FBCF08950E940B0A802D11F06BD0AA
:100E0000FACF089581E06DD015D080E86AC08FE7F1
:100E1000213039F08FEB223021F083E9233009F0C3
:100E200083ED810F0C94710788EE93E087D03197A2
:100E3000D9F7089583E0992781C08AEF90E00E9456
:100E40009E07A79AA69AA59AA49AA19AA09AA8984A
:100E500085E090E00E949E07A998AF98AE98AD9A61
:100E6000AC9AA99AEF93FF93E4ECF0E00E9492070A
:100E7000FF91EF91A9985FD0A99AEF93FF93E4ECCB
:100E8000F0E00E949207FF91EF91A99854D0A99A9F
:100E9000EF93FF93E4ECF0E00E949207FF91EF9153
:100EA000A99849D0AC98A99AEF93FF93E4ECF0E0AD
:100EB0000E949207FF91EF91A9983DD084E211D052
:100EC00089E00FD080E20DD088E20BD08EE009D00F
:100ED00086E007D00895A89A829505D004D02BD03B
:100EE0000895A898F9CF859510F4AC9A01C0AC98F4
:100EF000859510F4AD9A01C0AD98859510F4AE9A21
:100F000001C0AE98859510F4AF9A01C0AF98A99A28
:100F1000EF93FF93E4ECF0E00E949207FF91EF91D2
:100F2000A99808953197F1F70895689462F80895A3
:100F3000E89462F8089581E090E000C0EF93FF9399
:100F4000EE27E82BE92B31F0E0EDF7E03197F1F7F0
:100F50000197D1F7FF91EF9108958DE207FD8D93F1
:100F60008F2D881F802F881F8F57082F6894F7F8C0
:100F7000802F87FF15C080958395082F80E38D9380
:100F80008EE28D93802F815228F080E38D939927F4
:100F90009C93089544270A95802F09F196D01FC08D
:100FA000805230F09EE49D9381E48D939D93EFCF2A
:100FB0004427DF92EF92FF920F938FE1801B11F095
:100FC000082F83D089D09EE29D930F91FF90EF90E0
:100FD000DF9044270395003209F4D7CF2BD03F93FD
:100FE000EAE6F0E138E12F2D1E2D0D2DFF24EE2431
:100FF000DD244427000F111F221FA8F42F923F92D7
:101000000E940B0A102C0E940B0A202C0E940B0A33
:10101000302C0E940B0A3197410DD21CE31CF01CAE
:101020003F902F9001C0339631963A9519F73F9132
:1010300007D0AFCFDD0CEE1CFF1C0A95D9F7089541
:10104000002719E058D08F93802B11F0039501C031
:101050008F911A95B9F7802F882309F496CF8F9135
:10106000805D8D930A95D9F792CF0065CD1D80B232
:10107000E60E40597307A0ACB90350D6DC01286BCB
:10108000EE0094357700CA9A3B0065CD1D00B2E6AC
:101090000E0059730700ACB90300D6DC01006BEEFB
:1010A0000000357700009A3B0000CD1D0000E60EE1
:1010B000000073070000B9030000DC010000EE002F
:1010C0000000770000003B000000F694E794D794FE
:1010D00047950A95D1F7089500270DD08F93039572
:1010E0008F2D8E298D29842BC1F78F91805D8D9353
:1010F0000A95D9F74CCF1F930F93002710E2440FA6
:10110000DD1CEE1CFF1C001F802F9AE0890B10F0E5
:10111000082F43951A9599F7802F0F911F910895E5
:101120002093DD013093DE014093DF015093E00115
:1011300008952091DD013091DE014091DF01509151
:10114000E00108950E940B0A0D920020D9F708953E
:10115000D094E094F09491E0D90E9927E91EF91EFD
:1011600010950895D190E190F19001910895219109
:101170003191419151910895102F90E8FF0C001F7B
:101180000927990FF7941078652F90E8440F551FA1
:101190005927990F4795607800380895FF0C90E81B
:1011A0009027110F9795F794092F0895102FBD2CB4
:1011B000DE2CEF2CF02E11234AF4B094D094E0945E
:1011C000F0949FEFB91AD90AE90AF90A0EE1FF2053
:1011D00039F4FE2CED2CDB2CBB240850C2F76BC07D
:1011E00032F00A95BB0CDD1CEE1CFF1CF9CF01D0C0
:1011F000D5CFB7FE089590E8B91611F4D0FE089542
:101200009FEFD91AE90AF90A09F403950895DD92C6
:10121000ED92FD920C930895502F2D2D3E2D4F2DC4
:10122000612F08952DEC3CEC4CEC5DE366270FC07C
:1012300099DFF2DFDD24EE2490E8F92E0FE307C0FA
:1012400096DF05C02227332740E251E46627552365
:1012500051F1002381F190DF71F1162700585058A9
:101260000894050B18F407FD03C025C007FD23C033
:10127000469537952795F694E794D79422D0FF208A
:101280002AF0DD0CEE1CFF1C015073F09D2D96958D
:1012900048F0DD203AF4EE202AF491E0D90E9927A7
:1012A000E91EF91E7BCF07C09FE7092FF92A9FEFA0
:1012B000D92EE92E0895DD24EE24FF2400271127DE
:1012C00008959F929924AA24BB2488E1D216E306AC
:1012D000F40628F0D21AE30AF40A089401C08894AC
:1012E000991CAA1CBB1CDD0CEE1CFF1C8A9571F717
:1012F000D92CEA2CFB2C9F9008953EDFE1F2503868
:10130000D1F21627005850580894051F12F418F40B
:10131000CBCF08F0D0CF0AD0FF202AF0BB0CDD1CC9
:10132000EE1CFF1C3BCF0F5FFBF138CF9F9299243F
:10133000AA24BB24992788E1990CAA1CBB1CDD1C9C
:10134000EE1CFF1C30F4920EA31EB41ED91EE91E23
:10135000F91E8A9589F79F90089509DF0DDF5038AF
:1013600029F090E869270CC00AF045D017CF5FE359
:1013700022273327442701C0FADEFEDE5038B1F3BE
:10138000003899F3902F951B8BF312F434D0FACFD9
:10139000983118F0222733274427983028F0232F3C
:1013A000342F44279850F9CF992329F04695379543
:1013B00027959A95D9F7912F962742F014D0B0F639
:1013C000F794E794D7940F5F8BF66ECF10D051F05F
:1013D00008F4BEDEFF2052F2DD0CEE1CFF1C0150B3
:1013E000CBF762CF68CFD20EE31EF41E0895D21A57
:1013F000E30AF40A0895DF92EF92FF920F931F938E
:10140000D22EE32EF42E052F162F6F915F914F9160
:101410003F912F910895C895319600200895FBDFE4
:10142000D02CF9DFE02CF7DFF02CF5DF002D08954C
:10143000F2DF202DF0DF302DEEDF402DECDF502DE0
:10144000089507FB00680EF40F7757FB50680EF401
:101450005F7707FD02C057FF05C0D216E306F4060A
:10146000050708952D153E054F05500708950024E2
:101470000D280E280F28002A0020089591E005C0AD
:1014800092E003C094E001C098E0C5DF0D929A9508
:10149000E1F7089591E0882321F08894991F8A95B7
:1014A000E9F7892F90950895BB270E944A0A9C91DD
:1014B00098279C933197F1F798279C930895992743
:1014C0008D9193958823E1F7939511968C931197BD
:1014D0008E919A95D1F70895EA2FFB2F00244C9115
:1014E0008D9103948E32E1F711248D91139488230A
:1014F000E1F71A94101640F41197202F2119239523
:1015000080E38D932A95E9F7113039F59927AE2FAD
:10151000BF2FA00DB91FA00FB91F8C919C938533CD
:1015200008F421C031E08E918E32E9F38D3241F022
:10153000830F8A3319F480E331E001C033278C93A1
:10154000AE1789F7332341F0AE2FBF2FB8DF81E309
:101550004D3209F43196808308958827E00DF81FF5
:10156000E00FF81F80830895040F151F261F371FF3
:10157000089504171507260737070895000F111F50
:10158000221F331F089500951095209530950F5F09
:101590001F4F2F4F3F4F0895019110810EC00191B1
:1015A0001191219130810BC00191108117FF05C06D
:1015B0003FEF2FEF04C0008111272227332737FF89
:1015C00003C0E1DF8DE28D93CF93DF93CF92DF9263
:1015D000EF92AA24BB24CC24DD24EE2440E2CAE00E
:1015E000DD2755E093E38881890F87FD9F7083FD98
:1015F000907F891B89935A95A9F7C0DFAA1CBB1C51
:10160000CC1CDD1CEE1C4A9551F7E894EFE0FF2757
:1016100082910ED0EB30E0F71EF068948A2D0CD04A
:1016200088278D93EF90DF90CF90DF91CF91089531
:10163000982F829501D0892F8F70805D26F080339E
:1016400009F4089568948D93089541E003C042E041
:1016500001C044E0E40F8827F81F8291982F8295FB
:1016600006D0892F04D04A95C1F70C943E0B8F7099
:101670008A3008F0895F805D8D93089588278D9367
:10168000089581918D938823E1F7089594E08191E5
:101690008D939A95E1F7089509919191992351F0CD
:1016A0008A95D9F7319781918D930A9519F08823FE
:1016B000D1F70895E3CF8FEF83959D919923E1F7BB
:1016C000089550DD59DD0395AAF087E1DD0CEE1C8D
:1016D000FF1C8A9589F00A95CAF7FF205AF000246A
:1016E0000D280E280F28002039F00A95DD0CEE1C7D
:1016F000FF1CDAF70A9552CDDECDDDCD33DD0023B8
:10170000E2F3B5DE19F4D0DD0068089585E0C5D0B8
:10171000FF0C001F04830FE70695F794DDD0506897
:101720002CDE75DD139721E438E743ED5BEBE5DD57
:1017300027E831ED43E15DE399D02EE03CE343EC53
:101740005DEB94D022E83DEA4BE25EE38FD02CEED5
:1017500032E846E75EEB8AD020E931EE49EA5EE303
:1017600085D020E83FEE4FEF5EEB80D024EC3FEFDA
:101770004FE75FE37BD04BDD139784818F5799F060
:101780002AF4D82E0FEFE02EF02E04C0D82EEE242F
:10179000FF2400270BDD28E132E741E35FE3ADDD05
:1017A000E6DC3497EADD86C07FDD84C0DBDC86E0E2
:1017B00074D005830F772BE33AEA48EB5FE39DDDB6
:1017C00026DD139741D028F4858188236AF773DDDD
:1017D00071C08F778483C6DC349774DF18DD13976C
:1017E00023E632E446E357EB88DD29ED37EA4AE1A8
:1017F00059E33CD026E538E14EEA5AEB37D026E5EE
:101800003CE84DE15CE332D02DEC37E543E65DEB9F
:101810002DD02DEE3DEF45E75EE328D028E132E7FD
:1018200041E35FEB23D058D0A8DDF6DCDD24EE24C5
:10183000FF2404818FE7080F0695F79408DD858162
:10184000881F08F4F6DC36C097DC8827039512F46D
:101850008894089507301AF0812F08940895FF1C8A
:10186000881F0A95E2F7812B8894089586DD7FDC36
:10187000349743CDFCDD81F00F930F772F933F9387
:101880004F935F933CDF5F914F913F912F9135DDF7
:101890008EDF8F918078082B08950FB6F8944A92C6
:1018A0005A92E42DF52DA42DB52D480E8827581EEB
:1018B0000FBE08950FB6F894599049900FBE089541
:1018C00051DC802FFF0C001F901728F4091B881F84
:1018D0000795F7940895EFCC5FE340E8332722277C
:1018E0000895E9CC3FDC0023E2F3D9F388E0D5DFAB
:1018F0008EDC1196FF0C001F8FE7080F0795F794F9
:101900000695F79483E08F9387DC81DC13972ADCBC
:101910009EDC2DDC389731DD91E0D3DF8F918A9505
:1019200011F08F93F1CFC6CFD773A3456616A544A8
:10193000EC51383F9A9919400000ED4300B035450D
:101940009A99193F14AE473F14AEC73F00000000FC
:1019500000002041000000400000803F2020527520
:1019600068722D556E697665727369740000740033
:1019700020202020202020426F6368756D00466182
:101980006368646964616B74696B2050687973691A
:101990006B002020204750532D53696D756C617486
:1019A0006F720000583D00006D00593D00005A3D27
:1019B00000004C313D004C323D004C333D00543D65
:1019C00000002F0047504747412C00002E30303098
:1019D0002C002C4E2C002C452C312C20392C312E57
:1019E000302C203134322E312C4D2C34372E352CE6
:1019F0004D2C2C30303030004750524D432C0000DD
:101A00002E3030302C412C002C452C002C002C3258
:101A100039313230362C2C2C410024002A00244746
:101A2000504753412C412C332C33302C32352C323F
:101A3000342C33312C30362C32312C30372C31369B
:101A40002C31302C2C2C2C322E302C312E302C31B1
:101A50002E372A3333002447504753562C332C312A
:101A60002C31312C30372C37392C3036392C333659
:101A70002C30362C35392C3037342C34302C323154
:101A80002C34382C3136392C34352C33312C34323B
:101A90002C3232342C33362A37300000244750475A
:101AA00053562C332C322C31312C32352C34322CF1
:101AB0003234302C33312C31362C33392C32393806
:101AC0002C33362C33302C32362C3132382C3339FF
:101AD0002C31302C31382C3035342C33312A3742EC
:101AE00000002447504753562C332C332C31312CD3
:101AF00032342C31352C3034322C32352C32332CDC
:101B000030372C3331312C31382C31332C30372CC9
:101B10003334312C2A3435004665686C6572000018
:00000001FF
